:0B08D200EF1FAC0670011E4C70F622F8
:1008AB008F118E108D0F8C0E780E74FF12088DE445
:0B08BB00FBFAF9F8C312087A70EE2275
:10080000C200E4F50CF50DE50D450C70097F507E36
:10081000C3FDFC1208ABE50DF4450C6006E50D4583
:100820000C7002B20030000A050DE50D700C050CCD
:100830008008E50D150D7002150C750A00750B1E6C
:10084000E4F508F509C3E50994FFE50864809480A0
:1008500050B5C3E509950DE50C6480F8E5086480A2
:10086000985004C2B58002D2B5AF0BAE0A1208D2BE
:0A0870000509E50970CF050880CBEB
:030000000208C62D
:0C08C600787FE4F6D8FD75812002080060
:10087A00EB9FF5F0EA9E42F0E99D42F0E89C45F0D4
:01088A00224B
:10088B007401FF3395E0FEFDFC080808E6CF2FF658
:10089B0018E6CE3EF618E6CD3DF618E6CC3CF62231
:00000001FF
